:020000040000FA
:0600000068EF10F0120091
:0608000068EF10F0120089
:06082A000200362100006F
:100830000002000020000000342100003E02000001
:0408400002000000B2
:0C0844005EEC09F0FB0EDBCFF3FFDB06DF
:10085000F35000090AE0ACEC09F0FA0E17EC0AF0CC
:10086000F3E1151CF1E1010E01D0000E8DEF09F04E
:100870005EEC09F03B0EE12402E3E168E652E16E32
:10088000010EDB6A020EDB6AF90EDBCFF6FFFA0E11
:10089000DBCFF7FFFB0EDBCFF8FF0800F550DF6E74
:1008A000DF5002E1B1EF08F0250EDF5C02E0A4EFBB
:1008B00008F0030EDB6A040EDB6A050EDB6A060E27
:1008C000DB6A070EDB6AC6EC08F02D0EDF5C0CE07D
:1008D0002B0EDF5C09E0200EDF5C06E0230EDF5C00
:1008E00003E0300EDF5C1AE1DF50300A14E0130A37
:1008F0000FE0030A0AE00B0A05E0060AE4E1030E32
:10090000DB80E1D7030EDB82DED7030EDB84DBD78F
:10091000030EDB86D8D7030EDB88D5D72A0EDF5C23
:100920001BE1C2EC08F010EC09F010E0030EDB80D4
:1009300008680968130EDBCF0DF0140EDBCF0EF044
:1009400089EC0FF0040E06C0DBFF03D0130EF9ECA8
:1009500008F0C6EC08F00BD0090EDB6A67EC09F072
:1009600003E0DBEC09F0FAD7090EF9EC08F0030E0E
:10097000DBB0DB982E0EDF5C1BE1C6EC08F02A0E24
:10098000DF5C0BE1C2EC08F010EC09F003E1130EA0
:100990004BEC09F0C6EC08F00BD0090EDB6A67ECF3
:1009A00009F003E0DBEC09F0FAD7090E4BEC09F093
:1009B000680EDF5C07E1C6EC08F0680EDF5C1DE145
:1009C000030E18D0740EDF5C17E07A0EDF5C14E0C3
:1009D000480EDF5C06E0540EDF5C03E05A0EDF5C7D
:1009E00002E1020E07D06C0EDF5C03E06A0EDF5CF2
:1009F00004E1010E9EEC09F0C9DBDF506E0A01E153
:100A00007FD31E0A01E192D1200A01E18FD13F0A72
:100A100001E149D11A0A01E146D10D0A01E143D1B0
:100A2000200A01E140D13A0A01E13DD1200A01E169
:100A30003AD1260A01E135D10D0A01E132D11A0A73
:100A400001E1D9D0200A4AE0300A1FE0460A0EE050
:100A5000250A01E083D3D950F90FE96EFF0EDA20A1
:100A6000EA6E010EEE5E000EEE5AEE5AACEC09F0A4
:100A7000250EE66E95DB03E1151C01E169D3A8ECB8
:100A800009F001E26BD3DB2A69D3080EDB6A040E9E
:100A9000DB50010806E2040EDB0470EC09F0DB50C9
:100AA0008BDB080EDB5009E0030EDB50010B05E188
:100AB00072DB01E04DD3080EDB6A64DBEFCFDFFFB2
:100AC00020EC0AF003E1151C01E142D3A8EC09F087
:100AD00001E3DB2A60DB01E141D33AD3070EDB50AF
:100AE00002080FE1ECEC09F0030EB3EC09F00E0E76
:100AF000EECFDBFF0F0EEECFDBFF100EEECFDBFFF6
:100B000020D0F70EDBCF17F0F80EDBCF18F0020E77
:100B1000175E000E185AF70E17C0DBFFF80E18C04C
:100B2000DBFF17C0E9FF18C0EAFFA3EC09F0166A63
:100B30000E0E14C0DBFF0F0E15C0DBFF100E16C02B
:100B4000DBFF0E0EDBCFE6FF0F0EDBCFE6FF100E56
:100B5000DBCFE6FF06EC0FF0E552E552E552130E4F
:100B600007C0DBFF140E08C0DBFF060EDB5005E0FC
:100B7000130EE7EC09F001E26ADB0BEC0AF002E28B
:100B8000130E37DBCEEC09F006E0040EE7EC09F0BB
:100B900002E2050E2EDB030EDBB005D0FCDA01E02D
:100BA000D7D2080EDB6A090EDB6A0E0EDBCFF6FF2A
:100BB0000F0EDBCFF7FF100EDBCFF8FF0800F5506C
:100BC000DF6EDF5014E011EC0AF011E220EC0AF0C5
:100BD00003E1151C01E1BCD2BBDB01E3DB2A090EFA
:100BE000DB2AD9500E0FE96E000ECBDBE7D7D3DA44
:100BF00001E1B4D2ADD2C6DA110EEECFDBFF120E98
:100C0000EDCFDBFF110EDBCFE6FF120EDBCFE6FFF1
:100C1000F8EC0EF0E552E552130EF3CFDBFF140EA5
:100C2000F4CFDBFF060EDB5004E0130ED0DB01E255
:100C30000EDB0BEC0AF002E2130EDBDAAFDB05E0B1
:100C4000040EC5DB02E2050ED4DA030EDBB005D0DC
:100C5000A2DA01E07DD2080EDB6A090EDB6A110E12
:100C6000DBCFE9FF120EDBCFEAFFEFCFDFFFDF5074
:100C700014E0D7DB12E2E4DB03E1151C01E168D2EA
:100C800067DB01E3DB2A090EDB2A110EDB2ADBCF4F
:100C9000E9FF120EE8E3DB2AE6D77DDA01E15ED256
:100CA00057D2030EDB8E070EDB0410E195DB040E3A
:100CB0005ADB0A0EEECFDBFF0B0EEECFDBFF0C0E86
:100CC000EECFDBFF0D0EEECFDBFF6CD0070EDB505F
:100CD00003082CE1030EDBAE0DD0B2DA020E76DA99
:100CE000EFCF14F0156A166A176A14AE39D015687A
:100CF000166835D0F70EDBCF15F0F80EDBCF16F007
:100D0000020E155E000E165AF70E15C0DBFFF80E28
:100D100016C0DBFF15C0E9FF16C0EAFFEFCF14F0E5
:100D20000A0E14C0DBFF0B0EDB6A38D0070EDB5057
:100D3000020809E1030EDBAE04D059DB16AE10D079
:100D40000ED055DB0DD0030EDBAE12D079DA020ED9
:100D50003DDAF9DA166A176A15AE02D01668176816
:100D6000E2DA0C0E16C0DBFF0D0E17C0DBFF1AD047
:100D7000F70EDBCF16F0F80EDBCF17F0020E165E83
:100D8000000E175AF70E16C0DBFFF80E17C0DBFF78
:100D900016C0E9FF17C0EAFFD6DAC5DA0C0EDB6A27
:100DA0000D0EDB6A060EDB5005E1010EF36E050E3B
:100DB000F3CFDBFF150EDB6A160EDB6AD950370F57
:100DC000146E000EDA20156E390E14C0DBFF3A0ED9
:100DD00015C0DBFF380EDB6A080EDB6A0A0EAEDADE
:100DE000DF50780A12E0200A10E0280A0CE0200AFE
:100DF0000AE03F0A06E00D0A02E0200A08E1020EBE
:100E000005D0080E03D0080EDF26100E97DA030E69
:100E1000DBBE02D0DB92DB94DB50800B24E08ADA6D
:100E2000D890030EEB50000A08E6000EEE5C000EB0
:100E3000EE58000EEE58000EEE5815E213DA0B686D
:100E40000C680D680E68C0EC0EF00A0E02C0DBFFE5
:100E50000B0E03C0DBFF0C0E04C0DBFF0D0E05C044
:100E6000DBFF2D0E08D0030EDBA202D02B0E03D029
:100E7000DBA408D0200EF36E170EF3CFDBFF150EA8
:100E8000DB2A02D0170EDB6A050EDB5003E1B7D96F
:100E900001E189D01E0E146E210E156E000E166E25
:100EA000070EDBCF17F0186A196A1A6A17C00BF021
:100EB00018C00CF019C00DF01AC00EF0D3D9DCEC3C
:100EC0000FF014500224F36E15500320F46E1650E8
:100ED0000420F86EF4CFF7FFF3CFF6FF0800090EF9
:100EE000F5CFDBFF580EDF5C0FE1610EF36E090EEC
:100EF0007BD90AE3200E146E090EDBCFE7FF1450F6
:100F0000E75E090EE7CFDBFF070EDBCF14F0156AB3
:100F1000166A176A0FDA14C00BF015C00CF016C071
:100F20000DF017C00EF0EECF06F0EECF07F0EECFCB
:100F300008F0EFCF09F0DCEC0FF009C0EDFF08C0BE
:100F4000EDFF07C0EDFF06C0EFFF390EDBCFE9FF75
:100F5000DB063A0EDBCFEAFF01E2DB06090EDBCF50
:100F6000EFFF150EDB2A4BD995E1030EDBA61DD052
:100F70006F0EDF5C06E1C1D918E3150EDB285BDAE2
:100F800014D0780EDF5C09E0580EDF5C06E0620EDC
:100F9000DF5C03E0420EDF5C08E1020EF36E160E2A
:100FA000F3CFDBFF02D0150EDB6A030EDB50100B14
:100FB0000EE0040EDBCF14F0050EDB50D880145485
:100FC00006E2060EDB5003E1040EDB5034DA95D95D
:100FD0000AE2050EDBCFE7FF150EDB50E75E050EDC
:100FE000E7CFDBFF02D0050EDB6A040EDBCF14F087
:100FF000160E45D9D880145414E2160EDBCFE6FF46
:10100000150EDBCFE6FF040EDBCFE6FF050EDB504F
:10101000E552E75CE552D880E754E552D880E754C2
:101020005FD9030EDB50010B0BE1080EDB5008E02B
:10103000B2D801E08DD0080EDB50BED8080EDB6AB6
:10104000170EDB5007E088D9170EF1D903E1151C04
:1010500001E17ED0160EDB5016E07ED9300EE66E32
:101060009FD802E1151C74E077D9DFCFE6FF7EEC54
:101070000EF0E552E552E552F4CF15F00001F31CF5
:1010800002E1151C65E0050EDBCF14F0160EDB50F7
:10109000D880145409E2050EDBCFE7FF160EDB50B3
:1010A000E75E050EE7CFDBFF300EE66E050ECBD90F
:1010B0004FE1390EDB2ADBCFE9FF3A0E01E3DB2AF1
:1010C000DBCFEAFF090EEFCFDBFFDB500EE044D9A8
:1010D000090EADD902E1151C3BE0390EDB2ADBCF4E
:1010E000E9FF3A0EEDE3DB2AEBD755D831E1160ED6
:1010F000DBCFE6FF080EC3D8E552E7245DD82ED03B
:10110000070EDB50030A1CE0010A14E0030A07E0A3
:101110007BD9DBCFEEFF020EDBCFEDFF1FD0F5D882
:10112000196A17AE02D0186819682CD8BCD819C033
:10113000EEFF14D0EAD817BE186824D8B4D80ED061
:1011400063D9DBCFEFFF0AD07BD905E1151C03E1A2
:10115000F368F46810D0FCD801E3DB2A79D94DEFAD
:1011600004F0010EDBCF14F0020EDBCF15F014C03B
:10117000F3FF15C0F4FF3B0EE15C02E2E16AE552C9
:10118000E16ECBD029D9020EB3EF09F061D9080086
:10119000F550DF6E1200200EE66E080E23EF0AF007
:1011A0007EEC0EF0E552E552E552F3CF14F0F4CFA9
:1011B00015F00001F31C1200146E156AD950010FCE
:1011C0004DD91450EE261550ED221200185E000E77
:1011D000195AF70E18C0DBFFF80E19C0DBFF18C054
:1011E000E9FF19C0EAFF1200DBCFF4FFF350F45C13
:1011F0001200DB50E76E040EE7CFDBFF12000A0E91
:10120000DBCF14F00B0EDBCF15F00C0EDBCF16F09E
:101210000D0EDBCF17F0145015101610171012001A
:10122000130EEECFDBFF140EEDCFDBFF130EDBCF83
:1012300014F0140EDBCF15F00001800E151412000F
:10124000F70EDBCF18F0F80EDBCF19F01200050E09
:10125000DB50E66ED950130F01D9E552E750EE6E20
:10126000ED6A12000A0EDBCF06F00B0EDBCF07F0A3
:101270000C0EDBCF08F00D0EDBCF09F01200DBCF38
:10128000E6FF150EDBCFE6FF050EDB50E552E72447
:10129000E552E7241200DB50CED8010EF36E060EA5
:1012A000F3CFDBFF1200EE50EFCFEAFFE96E16C07E
:1012B000EEFF17C0EEFF18C0EEFF1200D9CFE6FF19
:1012C000DACFE6FFE1CFD9FFE2CFDAFF1200DFCFBE
:1012D000E6FFE66A36EC10F0E552E552F3501200F4
:1012E000E76E080EE7CFDBFF1200EECF14F0EECF73
:1012F00015F0EFCF16F0176A1200050EDBCF14F0D1
:10130000150EDB50D88014541200010EDBCF16F0FE
:10131000020EDBCF17F0186A1200E552E5CFDAFFB4
:10132000E7CFD9FF12000A0E14C0DBFF0B0E15C069
:10133000DBFF1200D9500A0F2EEF0AF0F36E070EF2
:10134000F3CFDBFF1200EECF14F0EFCF15F0120059
:10135000010EDB2A020E1200FC0EDBCFE6FFFD0EB3
:10136000DBCFE6FF1200145E000E155AF70E14C014
:10137000DBFFF80E15C0DBFF14C0E9FF15C0EAFF64
:101380001200DA20EA6EEF2AEECFF6FF000EEF220F
:10139000EECFF7FFEF22EECFF8FF1200040EDBCF07
:1013A000E6FF130EDB50E552E75C9ADFDB5004DF0B
:1013B000060EDB501200090EDB500A0DF350DF243D
:1013C000D00FE76E090EE7CFDBFFC6EF08F0DB506A
:1013D000F36E050EF4EF08F0F70EDBCF14F0F80E05
:1013E000DBCF15F01200DFCFE6FFD0EF08F028DFEB
:1013F000030EECDE75EF09F022EC04F0E552E55245
:10140000E552E55200091200BDDEEE50EFCFEAFFD3
:10141000E96E010E1200130EDB50F36E040EF4EFB2
:1014200008F0040EDB50F36E090EF4EF08F0DBCF8A
:10143000E6FFD0EF08F0E76E050EE7CFDBFF120006
:101440008BDFF3EF09F0DBCFE6FF86DFFCEF09F07F
:10145000D950F90FE96EFF0EC1EF09F0E96E000EE9
:06146000DA20EA6E120022
:0A146600D9CFE6FFE1CFD9FF040E55
:10147000E126DE6ADE6ADE6ADD6ADD52DD52FD0EDD
:10148000DBCF14F0FE0EDBCF15F0166A176A15AE2F
:1014900002D016681768D9CFE9FFDACFEAFF030E4A
:1014A000EB501718E8AE02D0173408D01450EE5C99
:1014B0001550EE581650EE581750EE580FE20C0E1D
:1014C000E66E48EC10F0E552D9CFE9FFDACFEAFF3B
:1014D000EE2A000EEE22EE22EE22D1D7040EE15CBF
:1014E00002E2E16AE552E16EE552E7CFD9FF120070
:1014F0000F0EC16E070EB46E936A300E926E0F0E11
:10150000946EF19E1200D9CFE6FFE1CFD9FF020E13
:10151000E1268250020B01E0010E080DF3CF16F018
:101520008250010B040DF3CF15F08050200B01E029
:10153000010EE824146E8050100B01E0010E1424FB
:1015400015241624DE6EDD6ADECF14F0DDCF15F033
:1015500014C0F3FF15C0F4FF020EE15C03E200D0FB
:10156000E16AE552E16EE552E7CFD9FF12008092C1
:10157000320EE66E84EC10F0E5528084320EE66E98
:1015800084EC10F0E5528094320EE66E84EC10F09C
:10159000E55212008082320EE66E84EC10F0E552C5
:1015A0008084320EE66E84EC10F0E5528094320EA8
:1015B000E66E84EC10F0E5521200380E816ED7DF33
:1015C000320EE66EE66A4FDFE552E552010E816E9D
:1015D000CEDF320EE66EE66A46DFE552E5520D0ECC
:1015E000816EC5DF320EE66EE66A3DDFE552E552FA
:1015F000060E816EBCDF320EE66EE66A34DFE5521F
:10160000E5521200010E816EB2DF0A0EE66EE66A46
:101610002ADFE552E5521200D9CFE6FFE1CFD9FF2C
:10162000020E816EA4DF0A0EE66EE66A1CDFE5524A
:10163000E552FD0EDBCFE6FFFE0EDB50280DF3502A
:10164000E552E724E76EFE0EE7CFDBFFFD0EDB6A17
:10165000FE0EDB50F36EFD0EDBCFF4FFF350F45CB7
:101660000BE2140E816E83DF320EE66E84EC10F016
:10167000E552FD0EDB2AECD7E552E7CFD9FF120089
:10168000D9CFE6FFE1CFD9FFFE0EDB50816E82DFBE
:10169000320EE66E84EC10F0E552E552E7CFD9FF4A
:1016A0001200D9CFE6FFE1CFD9FFFD0EDBCFE9FF76
:1016B000FE0EDBCFEAFFEF500EE0FD0EDBCFE9FFC1
:1016C000DB2AFE0EDBCFEAFF01E3DB2AEF50E66EFA
:1016D000D7DFE552EAD7E552E7CFD9FF1200020182
:1016E000246B300E926EF00E936EEF0E206F20C2C0
:1016F00081FF040E216F2151000821E22051FE0BD1
:10170000E842206F20C281FF050EE66EE66AABDE7E
:10171000E552E5528150100B09E08150200B06E0A4
:101720008150400B03E08150800B01E10AD8020197
:10173000240502E1255104D02105216FDCD7CFD744
:101740001200F00E936E81CF23F202012315226F57
:101750000F0E2015206F20512211206F81CF23F210
:10176000F00E2315226FF00E225D01E0F7D7936A89
:1017700006D826C225F20201010E246F12000201D2
:10178000276B100E275D14E22751EA6A000FE96EFD
:10179000020EEA22EF50205D08E12751EA6A100F9D
:1017A000E96E020EEA22EFCF26F22729276FE9D74A
:1017B00026C281FF640EE66EE66A55DEE552E5520A
:1017C00012000201286B070E285D1DE288DF02016E
:1017D000296F2851EA6A2A0FE96E020EEA2229C20D
:1017E000EFFF2851EA6A2A0FE96E020EEA22EF5053
:1017F000460802E108D004D029C2E6FF41DFE552E5
:101800000201282BE0D72851EA6A2A0FE96E020E5E
:10181000EA22EF6A12000201286B070E285D16E229
:101820002851EA6A2A0FE96E020EEA22EF50E66EAC
:1018300027DFE55202012829EA6A2A0FE96E020E23
:10184000EA22EF5001E102D0282BE7D71200D9CFCE
:10185000E6FFE1CFD9FFE652F250800B01E0010E26
:10186000DF6EF29EA69EA69CA684FE0EDB50A96E9D
:10187000FD0EDB50A86E550EA76EAA0EA76EA682AF
:10188000A6B2FED7A694DF50E8B0F28EE8A0F29E92
:10189000E552E552E7CFD9FF1200D9CFE6FFE1CFFD
:1018A000D9FFA69CA69EFE0EDB50A96EA680A8506E
:1018B00000D0E552E7CFD9FF12004D0EE66EE66A82
:1018C0006C0EE66E39EC0EF0E552E552E552120070
:1018D000D9CFE6FFE1CFD9FF040EE126DE6ADE6A4A
:1018E000DE6ADD6ADD52DD52D9CFE9FFDACFEAFFE9
:1018F000D890030EEB50000A08E6400EEE5C0D0E89
:10190000EE58030EEE58000EEE5811E29EAA04D0D7
:1019100000EC10F00ED001D000D0D9CFE9FFDACF23
:10192000EAFFEE2A000EEE22EE22EE22DDD7000EB6
:1019300000D0146E040EE15C02E2E16AE552E16E51
:101940001450E552E7CFD9FF1200D9CFE6FFE1CF1F
:10195000D9FFE6529EAAFED700EC10F0DF6EDF50F2
:1019600000D0E552E552E7CFD9FF1200D9CFE6FF0C
:10197000E1CFD9FFE6529EAAFED700EC10F0DF6E51
:10198000DFCFE6FF1FEC10F0E552DF5000D0E5524C
:10199000E552E7CFD9FF120090DFA10E146E1E0EA4
:1019A000156E166A14C0E6FF15C0E6FF16C0E6FF06
:1019B000EDEC0DF0E552E552E552E80EE66E030E51
:1019C000E66E51DDE552E552D1DF0201386F396B29
:1019D000800B01E03969420E381901E139514AE1C1
:1019E000970E146E1E0E156E166A14C0E6FF15C013
:1019F000E6FF16C0E6FFEDEC0DF0E552E552E552CC
:101A0000830E146E1E0E156E166A14C0E6FF15C006
:101A1000E6FF16C0E6FFEDEC0DF0E552E552E552AB
:101A2000040EE66E330EE66E020EE66E5AEC0FF012
:101A3000E552E552E5520201376B330EE66E020EB7
:101A4000E66EB6EC0FF0E552E5524C0E0201355D44
:101A500012E1760E146E1E0E156E166A14C0E6FFA5
:101A600015C0E6FF16C0E6FFEDEC0DF0E552E552BD
:101A7000E55202D062D061D0620E146E1E0E156E59
:101A8000166A14C0E6FF15C0E6FF16C0E6FFEDECCF
:101A90000DF0E552E552E55202013A6B3B6B040E44
:101AA0003BAF02D0D89003D03A5D000E3B5913E211
:101AB0005DDF0201386F396B800B01E03969330E4D
:101AC0003A25E96E020E3B21EA6E38C2EFFF3A2B4F
:101AD000000E3B23E4D74F0E365D02E0000E01D02E
:101AE000010E166E520E355D02E0000E01D0010EA1
:101AF000156E4F0E345D02E0000E01D0010E146E23
:101B0000420E335D02E0000E01D0010E14141514D4
:101B1000161411E0560E146E1E0E156E166A14C0C1
:101B2000E6FF15C0E6FF16C0E6FFEDEC0DF0E5524E
:0C1B3000E552E55201D001D030D7120080
:041B3C002A0EF66E09
:101B4000080EF76E000EF86E00010900F550656F83
:101B50000900F550666F03E1656701D03DD00900CB
:101B6000F550606F0900F550616F0900F550626F24
:101B700009000900F550E96E0900F550EA6E090008
:101B800009000900F550636F0900F550646F090002
:101B90000900F6CF67F0F7CF68F0F8CF69F060C0C2
:101BA000F6FF61C0F7FF62C0F8FF0001635302E176
:101BB000645307E00900F550EE6E6307F8E264072E
:101BC000F9D767C0F6FF68C0F7FF69C0F8FF0001EA
:0A1BD0006507000E665BBFD7120028
:061BDA00D9CFE6FFDACFCF
:101BE000E6FFE1CFD9FFE2CFDAFFE652E652E65256
:101BF000E652D950FB0F146EFF0EDA20156E14C09A
:101C0000DEFFDD6EDECFE6FFDDCFE6FFFB0EDBCFD6
:101C1000E6FFFC0EDBCFE6FFFD0EDBCFE6FF3EC2AC
:101C2000E6FF3FC2E6FF38EC04F0146E070EE15CFD
:101C300002E2E16AE552E16E1450020EF3CFDBFFDF
:101C4000030EF4CFDBFF020EDBCF14F0030EDBCF6D
:101C500015F014C0F3FF15C0F4FF040EE15C02E2BE
:101C6000E16AE552E16EE552E5CFDAFFE7CFD9FF51
:021C7000120060
:0E1C7200D9CFE6FFDACFE6FFE1CFD9FFE2CF10
:101C8000DAFFAC6AAB6AFD0EDBB0AC88DBA202D037
:101C9000AC8CAB8CDBB4AC8EDBA602D0AB8801D0B5
:101CA000AB8ADBB8AC849E98DBBAAB86DBAC02D0E7
:101CB0009D8A01D09D9A9E9ADBAE02D09D8801D06C
:101CC0009D98FB0EDB50AF6EFB0EFC0EDBCF15F0CC
:101CD00015C014F0156A1450B06EAC8AAB8E949C8B
:101CE000948EAC50100B04E0AC50800B01E1948C4E
:0C1CF000E552E5CFDAFFE7CFD9FF120084
:041CFC00D9CFE6FF57
:101D0000DACFE6FFE1CFD9FFE2CFDAFFFB0EDBCF80
:101D100014F0FC0EDBCF15F00001800E15141AE153
:101D2000FB0EDBCFE9FFFC0EDBCFEAFFEECFF3FFCC
:101D3000EDCFF4FFEE2A000EEF22F3CFE9FFF4CF50
:101D4000EAFFFD0EDBCFEFFFEF50156AF36E15C013
:101D5000F4FF10D0FB0EDB50FE0806E1FD0EDBCFDA
:101D6000E6FF76EC10F005D0FD0EDBCFE6FF98EC39
:101D700010F0E552E552E5CFDAFFE7CFD9FF1200C8
:101D800006500B02F3CF02F0F4CF03F00C02F35035
:101D90000326000EF420046E06500D02F3500426B4
:101DA000000EF420056E06500E02F3500526075073
:101DB0000B02F3500326F4500422000E05220750B4
:101DC0000C02F3500426F450052207500D02F35084
:101DD000052608500B02F3500426F4500522085043
:101DE0000C02F350052609500B02F3500526120091
:101DF000FE0EE3CFE9FFFF0EE3CFEAFFF36AF46ADA
:101E0000EE5203E0F34AF42AFBD71200FF0EE3CFB1
:101E1000F8FFE552FF0EE3CFF7FFE552FF0EE3CFE9
:101E2000F6FFE552E66AE66AE66A0900F55209E05D
:101E3000FD0EE32A05E1FE0EE32A02E1FF0EE32A8E
:101E4000F4D7FD0EE3CF07F0FE0EE3CF08F0FF0E50
:061E5000E3CF09F01200CF
:0A1E560020484F4C4120424F524FEC
:101E600021000D0A5459504520574F524420424FEB
:101E7000524F0D0A3E0020484F4C4120414D4947EA
:101E80004F21000D0A5459504520574F52442048C5
:101E90004F4C410D0A3E002057454C434F4D4521C4
:101EA000000D0A54595045204C4554544552204287
:041EB0000D0A3E00D9
:0C1EB400D9CFE6FFDACFE6FFE1CFD9FF7F
:101EC000E2CFDAFFE652E652DF6AFB0EDB50DF5C60
:101ED00018E29EAAFED700EC10F0E76E010EE7CFE5
:101EE000DBFFFC0EDBCFE9FFFD0EDBCFEAFF010ECF
:101EF000DBCFEFFFFC0EDB2AFD0E01E3DB2ADF2A3E
:101F0000E4D7E552E552E552E5CFDAFFE7CFD9FF56
:021F10001200BD
:0E1F120009C013F008C012F008500D02F4CF01
:101F200007F0F3CF06F009500E02F4CF09F0F3CF1B
:101F300008F00D02F3500726F4500822E86A09223F
:101F400012500E02F3500726F4500822E86A0922C4
:101F50000EAEAFEF0FF01250085E1350095A13AED9
:0C1F6000000C0D50085E0E50095A000CD9
:041F6C00D9CFE6FFE4
:101F7000DACFE6FFE1CFD9FFE2CFDAFFACA2FED79E
:101F8000FC0EDBCFE9FFFD0EDBCFEAFFEF50E66E84
:101F90001FEC10F0E552FC0EDBCFE9FFDB2AFD0E53
:101FA000DBCFEAFF01E3DB2AEF50E8E1E552E5CFC2
:081FB000DAFFE7CFD9FF1200B0
:081FB800056A046A036A026A6B
:101FC000200EE76ED89006360736083609360236F8
:101FD0000336043605360B50025C0C5003580D5086
:101FE00004580E50055809E30B50025E0C50035A7A
:101FF0000D50045A0E50055A062AE72EE4D7120057
:10200000D9CFE6FFDACFE6FFE1CFD9FFE2CFDAFFA3
:10201000E652F20E00016A17ABAC03D06A91ABB086
:102020006A81ABB46A85ABB26A87AE50DF6EDF50AF
:0E203000E552E552E5CFDAFFE7CFD9FF120007
:02203E00D9CFF8
:10204000E6FFDACFE6FFE1CFD9FFE2CFDAFFACACB3
:1020500004D0AC9000016AB3AC80FD0EDB50AD6ED5
:0C206000E552E5CFDAFFE7CFD9FF120010
:04206C00F36AF46AB5
:10207000FF0EE124E96EFF0EE220EA6EED6607D066
:102080002F0EEF6404D03A0EEF6001D0F32A120055
:10209000FF0EE3501B6E480E01D04C0EE76EE72E8C
:1020A000FED7E76AE72EFED71B2EF7D700001200F7
:1020B000000EF36E00EE00F0080E01D81200EA6088
:1020C00002D0EE6AFCD7F350E9601200EE6AFCD74A
:1020D00012EE40F022EE40F0F86A019C9EEC0DF00A
:0C20E00099EC10F0CCEC0CF0FBD71200D7
:0420EC00FF0EE350B0
:1020F000ACBA04D0AF6AAB8EAC8A949CACA2FED7CB
:08210000AD6EF36EF46A1200EB
:08210800FF0EE350E84E120047
:0E211000000000D000D000D0E82EFAD7120058
:02211E0030315E
:0F212000323334353637383961626364656600AF
:0221300012009B
:02213200120099
:02213400FEFFAC
:0A213600EEEDEBE7DEDDDBD7BEBD0A
:10214000BBB77E7D7B773031323334353637383923
:06215000414243444546F4
:00000001FF
